:04002E0043B1402278
:0400460053B1BF22D1
:04004E0063B1402238
:0100320022AB
:01004A002293
:01005200228B
:0112FF0022CC
:0121EA0022D2
:10188600EF5407FE7401A806088002C333D8FCFE95
:10189600EF131313541FFFED601EEF14600E146058
:1018A6000F14601024037031EE428022EE42902223
:1018B600EE42A022EE42B022EF14600F1460111423
:1018C600601324037013EEF4528022EEF452902239
:0918D600EEF452A022EEF452B02F
:0118DF0022E6
:101BC800EF54F824F8601024F8601024F86010240A
:101BD80018700EAE80800AAE908006AEA08002AE6D
:101BE800B0EF5407FF7401A807088002C333D8FC7C
:0B1BF8005206EE60047F0180027F00B7
:011C030022BE
:10000E00E58012064B900001E59012065D9000020D
:0D001E00E5A012065D900003E5B002065D4E
:101E8600120605902861F0F58090000112061E905A
:101E96002862F0F59090000212061E902863F0F575
:0E1EA600A090000312061E902864F0F5B022F2
:101F0C0090286074FFF090285FF090285EF0902885
:101F1C005DF0902864F0902863F0902862F090288F
:031F2C0061F0223F
:1015FA00E4F5B2F5B3F5B4F5B590285DE0FF908057
:10160A0000F090285EE0FE908001F090285FE0FDF7
:10161A00908002F0902860E0FC908003F08FB28EF8
:10162A00B38DB48CB5902861E0F580A3E0F590A362
:10163A00E0F5A0A3E0F5B090285DE0F4908004F016
:10164A0090285EE0F4908005F090285FE0F49080A6
:10165A0006F0902860E0F4908007F075B1BF75B687
:02166A00442218
:102152008F568D57300603020FFBAD57AF56121044
:022162001A223F
:0121EB0022D1
:0121EC0022D0
:0D00360090286574FFF0A3F0A3F0A3F02262
:1016DD00E4F5B2F5B3F5B4F5B5902865E0FF90806B
:1016ED0000F0902866E0FE908001F0902867E0FD04
:1016FD00908002F0902868E0FC908003F08FB28E0D
:10170D00B38DB48CB5902869E0F580A3E0F590A376
:10171D00E0F5A0A3E0F5B0902865E0F4908004F02A
:10172D00902866E0F4908005F0902867E0F49080B2
:0C173D0006F0902868E0F4908007F0228D
:0121ED0022CF
:100CA400D204120B275003020DEE90E6B9E024EDB6
:100CB4007003020D9324E37003020DB6248E7003B7
:100CC400020DE7147003020DE724916003020DEC9A
:100CD400E490E68AF090E6BEE090E68BF090E6A021
:100CE400E020E1F9E4F5B2F5B3F5B4F5B590E744E5
:100CF400E090285DF0908000F090E745E090285E59
:100D0400F0908001F090E746E090285FF090800238
:100D1400F090E747E0902860F0908003F090E7447B
:100D2400E0F5B2A3E0F5B3A3E0F5B4A3E0F5B59024
:100D3400E740E0902861F0F58090E741E090286278
:100D4400F0F59090E742E0902863F0F5A090E74337
:100D5400E0902864F0F5B090E744E0F4908004F06B
:100D640090E745E0F4908005F090E746E0F4908049
:100D740006F090E747E0F4908007F090E6BAE025AB
:100D8400E025E05404FFE5B154FB4FF5B1805B90DE
:100D9400E740E5B2F0A3E5B3F0A3E5B4F0A3E5B50D
:100DA400F0A3E580F0A3E590F0A3E5A0F0A3E5B0FF
:100DB400802190E740E580F0A3E590F0A3E5A0F062
:100DC400A3E5B0F0A3E5B2F0A3E5B3F0A3E5B4F076
:100DD400A3E5B5F0E490E68AF090E6BEE090E68BF9
:0C0DE400F080071209868002D322C3228F
:100F2B0012010002000000400516048001000102BE
:100F3B0000010A0600020000004001000902200027
:100F4B00010100A0FA0904000002FF0000000705E0
:100F5B0002020002000705860200020009022000BF
:100F6B00010100A0FA0904000002FF0000000705C0
:100F7B00010240000007058102400000140300003D
:100F8B000000000000000000000000000000000056
:100F9B002603410043004300450053002000490055
:100FAB002F004F002000500072006F00640075008E
:100FBB0063007400730018035500530042002D00AA
:100FCB00440049004F002D0033003200490000005F
:100FDB00808182838485868790919293949596974E
:100FEB00A0A1A2A3A4A5A6A7B0B1B2B3B4B5B6B73E
:100FFB00C0D0C0E0EF900FDB93901012F0ED900F8C
:10100B00DB93901014F0A2009200D0E0D0D022C05D
:10101B00D0C0E0EF900FDB93901031F0ED900FDB31
:0F102B0093901034F0A200B39200D0E0D0D02206
:10209800564A616E20323520323031384031343A78
:0B20A80030303A35300000000000002E
:10212800021720AF02080000010F01010C01010A8B
:04213800010114FF8E
:1020B300902803E0FF7006902802E0600890280251
:0920C300E0FD0220291221DB22BC
:101F52007E007F6D7D007B017A2879001207359023
:101F62002800740AF0E4A3F0121F0C1215FA021FE3
:011F720093DB
:10200D007D021219DB902800E0B40A04A3E06003FE
:0C201D00021F527D6D1219DB1215FA2211
:101F9300902800740AF0E4A3F07A287B007D6D7F1B
:0F1FA300017E1F121D597D6D7F007E1F0221D808
:1017B4001220B390E6BEE0F535753702E535605783
:1017C400C3944050058535368003753640E490E671
:1017D4008AF090E68BE536F090E6A0E020E1F9E4AB
:1017E400F534E534C39536502574402534F582E448
:1017F40034E7F583E0FFAE370537EE7C007B012448
:1018040000F9EC3428FAEF12064B053480D4C3E512
:0A181400359536F53580A50220B3A6
:1012300090E6B8E030E745E4F52BF52AE52AC394BB
:101240000850247E007B01745D252AF9EE3428FACB
:10125000120605FF7440252BF582E434E7F583EF91
:10126000F0052A052B80D5E490E68AF090E6BEE0F2
:1012700090E68BF090E6A0E04480F02290E6BEE09D
:1012800090E68BF090E6A0E020E1F990E6BEE06405
:10129000086003C20422E4F52AF52BE52AC394086A
:1012A00050247440252BF582E434E7F583E0FFE514
:1012B0002A7C007B01245DF9EC3428FAEF12064BFE
:1012C000052A052B80D590E6BAE0B4CE08A3E0B499
:0512D000AC03121F93A6
:0112D50022F6
:0F219800D3E51A950EE519950D40031221A722E4
:0121EE0022CE
:101F2F00902805E0FE902804E07C002400F50EECDC
:101F3F003EF50D450E7007C28CC2A9C20522D28C88
:031F4F00D2A922F2
:0121EF0022CD
:101B080090E6BEE090E68BF090E6A0E020E1F9E4F4
:101B1800FF74422FF582E434E7F583E0FEEF7C00A2
:101B28007B012465F9EC3428FAEE12064B0FBF0846
:101B3800E090E740E0902804F090E741E090280525
:041B4800F0021F2F59
:0F21A7001216DDE4F512F513F519F51AD205221B
:101FD100C205E4F512F513F519F51AC28CC2A9531D
:0E1FE1008EF75389F14389011221EF021F2F61
:101C0400E50945086019E50915097002150814C3AA
:101C140094FFE50864809480501C120046801730BD
:101C240004147508057509FF12002EC204E4F512A8
:0B1C3400F513F519F51A300502D20473
:011C3F002282
:100DF00090E6B8E020E703020EA5E4F52B90280466
:100E0000E0FFAE2B052B74402EF582E434E7F5832A
:100E1000EFF0902805E0FFAE2B052B74402EF582F5
:100E2000E434E7F583EFF0E4F52AE52AC3940850AB
:100E3000247E007B017465252AF9EE3428FA120617
:100E400005FF7440252BF582E434E7F583EFF005C8
:100E50002A052B80D5AE2B052B74402EF582E43469
:100E6000E7F583E51AF0E519FFAE2B052B74402E4C
:100E7000F582E434E7F583EFF0A205E433FFAE2B0F
:100E8000052B74402EF582E434E7F583EFF0C205BC
:100E9000E490E68AF090E6BEE090E68BF090E6A063
:100EA000E04480F02290E6BEE090E68BF090E6A071
:100EB000E020E1F9C20590E6BEE0640A6003C204E6
:100EC00022E4F52BAF2B052B74402FF582E434E799
:100ED000F583E0902804F0AF2B052B74402FF582AA
:100EE000E434E7F583E0902805F0E4F52AE52AC329
:100EF000940850247440252BF582E434E7F583E010
:100F0000FFE52A7C007B012465F9EC3428FAEF1216
:100F1000064B052A052B80D5121F2F90E6BAE0B4A8
:0A0F2000CE08A3E0B4AC03121F9347
:010F2A0022A4
:0412FB00750F012248
:10181E001220B390E6BEE0F535E4F537E5356057B6
:10182E00C3944050058535368003753640E490E606
:10183E008AF090E68BE536F090E6A0E020E1F9E440
:10184E00F534E534C39536502574402534F582E4DD
:10185E0034E7F583E0FFAE370537EE7C007B0124DD
:10186E001BF9EC3428FAEF12064B053480D4C3E58D
:07187E00359536F53580A514
:011885002240
:10193700150FE50F704B90281BE0F50F1221EBE414
:10194700F55390285CE0FFE553C39F5031E55325DD
:10195700E0241CF582E43428F583E0F554E55325AB
:10196700E0241DF582E43428F583E0F555547FFD26
:10197700E555339206AF54122152055380C4122104
:01198700EC73
:01198800223C
:101F730090E6BEE090E68BF090E6A0E020E1F990D9
:101F8300E740E0902806F090E741E0902807F02230
:10156F00150CE50C60030215F9902806E0F50C7BCD
:10157F00017A28799F12000EE4FFFE749F2EF582E8
:10158F00E43428F583E0FD746D2EF582E43428F5FC
:10159F0083E06DF97D01E4FCECC394085046E95DEE
:1015AF00602974712FF582E43428F583E014F07408
:1015BF00712FF582E43428F583E07020746D2EF5D9
:1015CF0082E43428F583E06DF08000902807E0FB7B
:1015DF0074712FF582E43428F583EBF00CED25E0E0
:0A15EF00FD0F80B40EEE640470914D
:0115F90022CF
:1020CC0090E6BEE090E68BF090E6A0E020E1F9907F
:0820DC00E740E0902808F02223
:101C7C00E4F515FF74912FF582E43428F583E0FE2A
:101C8C00749B2FF582E43428F583EEF074912FF5D4
:101C9C0082E43428F583E0FE74972FF582E434282F
:081CAC00F583EEF00FBF04CC3C
:011CB400220D
:10174900150AE50A7064902808E0F50A7B017A28F1
:10175900799112000EE4FF749B2FF582E43428F589
:1017690083C083C082E0FE74912FF582E43428F5AA
:1017790083E0FDEE5DD082D083F074972FF582E48B
:101789003428F583C083C082E0FE74912FF582E48A
:101799003428F583E0FDEE4DD082D083F00FBF04ED
:0A17A900B6E515C394FF50020515C4
:0117B3002213
:0421D0007514FF2261
:10166C00E4F5580514F55890281AE0FFE558C39F87
:10167C005054E55825E0240BF582E43428F583E03A
:10168C00C39514501EE55825E0240AF582E434284D
:10169C00F583E0FE547FFFEE30E7047D0080207D73
:1016AC0001801CE55825E0240AF582E43428F583F2
:1016BC00E0FE547FFFEE30E7047D0180027D0012D6
:1016CC001886055880A1902809E0B51403E4F51498
:0116DC0022EB
:101DC20090E6BEE090E68BF090E6A0E020E1F9E438
:101DD200FF74402FF582E434E7F583E0FEEF7C00E8
:101DE2007B012409F9EC3428FAEE12064B0FBF12DC
:011DF200E010
:011DF30022CD
:0413B8008E348F35AB
:1013BC00E4F536E53564024534700C90E741F0E510
:1013CC0035153570021534E53564014534701690C9
:1013DC00E740746DF090E6BEE090E68BF0E53515D5
:1013EC003570021534E5354534605D90E6A0E0209B
:1013FC00E1F9C3E5359440E53494005004AD3580F3
:10140C00027D40E4FFEFC39D5025AE360536EE75E8
:10141C0083007B012400F9E5833428FA120605FECB
:10142C0074402FF582E434E7F583EEF00F80D6E4B8
:10143C0090E68AF090E68BEDF0FFC3E5359FF5352D
:08144C00E5349400F534809DA5
:011454002275
:1000560090E6B8E030E76390E6BFE0FE90E6BEE0EB
:10006600FDEDFF4E7002804D90E6BDE0FD90E6BCD2
:10007600E04D70030213B890E6BDE060030203EBA7
:1000860090E6BCE01460030203EB7537FF75382079
:10009600753998753A00753B1E7B017AE7794112EE
:1000A60019897B017AE7794012213DEF0490E740F8
:1000B600F090E6BEE090E68BF02290E6BFE0FF907F
:1000C600E6BEE04F707790E6BDE0704D90E6BCE08E
:1000D60024EF6023249F603024FD603324F36034D2
:1000E6002472703590E6BAE064CE702DA3E064AC5D
:1000F6007027121F93802290E6BAE0B4CE1BA3E0CD
:10010600B4AC16121F528011E490281AF0800A75BA
:1001160014FF8005E490285CF090E6BDE064806002
:10012600030203EB90E6BCE0640160030203EB907C
:10013600E6BAE0902802F090E6BB02020590E6BF20
:10014600E060030203EB90E6BDE0FE90E6BCE07CD7
:10015600002400FFEC3EFEEF8EF012070801AB0014
:100166002001AB002101AB002201AB002301E0001E
:100176002F020D0041021B005102290053024900C3
:100186006102570063027700710285007302A500C1
:100196007402FB0081030900830329008403808025
:1001A60001000003EB90E6BEE0B46B031217B490B7
:1001B600E6BCE030E0031215FA90E6BCE020E1036D
:1001C6000203EB90E6BAE064CE60030203EBA3E021
:1001D60064AC60030203EB021F9390E6BEE0640288
:1001E60060030203EBE090E68BF090E6A0E020E1EE
:1001F600F91220B390E740E0902802F090E741E042
:10020600902803F00203E890E6BEE0640A60030269
:1002160003EB021B0890E6BEE0640260030203EBF8
:10022600021F7390E6BEE0640160030203EBE090F8
:10023600E68BF090E6A0E020E1F990E740E0902818
:1002460006F02290E6BEE0640160030203EB0220A2
:10025600CC90E6BEE0640160030203EBE090E68B1F
:10026600F090E6A0E020E1F990E740E0902808F061
:100276002290E6BEE0641260030203EB021DC29008
:10028600E6BEE0640160030203EBE090E68BF090CB
:10029600E6A0E020E1F990E740E0902809F02290FE
:1002A600E6BEE0640260030203EB90281AE0C39402
:1002B6000840030203EB90E6BEE090E68BF090E682
:1002C600A0E020E1F990E740E0FF90281AE0FE2543
:1002D600E02408F582E43428F583EFF090E741E066
:1002E600FFEE25E02409F582E43428F583EFF0904B
:1002F600281A02037C90E6BEE0644260030203EB28
:1003060002181E90E6BEE0640160030203EBE09073
:10031600E68BF090E6A0E020E1F990E740E0902837
:100326001BF02290E6BEE0640260030203EB902815
:100336005CE0C3942040030203EB90E6BEE090E647
:100346008BF090E6A0E020E1F990E740E0FF9028EE
:100356005CE0FE25E0241AF582E43428F583EFF00C
:1003660090E741E0FFEE25E0241BF582E43428F512
:1003760083EFF090285CE004F02290E6BEE090E681
:100386008BF090E6A0E020E1F990E6BEE064047010
:010396005412
:1003970090E740E0FCA3E0FDA3E0FEA3E0F52D8E8F
:1003A7002C8D2B8C2AFBAA2CA92BA82A7F007E1B1D
:1003B7007D377C4B1204E78F318E308D2F8C2EAB1F
:1003C70031AA30A92FA82EE4FFFE7D807C471203B7
:1003D700EF1205848E328F33EF902802F0E532A3B7
:0403E700F01220B33D
:0103EB0022EF
:10207D0090E6047480F00000007402F0000000741B
:0B208D0006F0000000E4F0000000225C
:0121F00022CC
:101B4C00E4F5257AE779407F40AB077D087FF87E86
:101B5C001D1219E3E4F52574402525F582E434E7DC
:101B6C00F583E0FDE52575F002A42489F9740F35A1
:0E1B7C00F08982F583EDF00525E525B408D942
:011B8A002238
:101C400090E678E05410FFC4540F4450F51013E4AC
:101C500033F516438E201200321221C8121B4C128B
:101C6000004AD20012200D121FD11212FB121C7C4E
:0C1C70001221D01220B3120046020052D4
:101FEF001212FF121C04122198E5B190E68020E72F
:0E1FFF0006E04408F08004E054F7F00221EA06
:0618E0008B1B8A1C891D10
:1018E600E4F51E12213D8F1FE51F25E02402900F0F
:1018F600C1F0E4F51EAF1FEF3395E0FEC3E51E9F72
:10190600EE6480F87480985027AB1BAA1CA91D852D
:101916001E8275830012061EFDE51E75F002A424C4
:10192600C3F9740F35F08982F583EDF0051E80C585
:01193600228E
:061A77008E3A8F3BAC0526
:101A7D00E4FDE5166012E53AFF7E000DEE2518F542
:101A8D0082E43517F583EFF0AE050DE5182EF582DE
:101A9D00E43517F583E53BF0AF050DE5182FF5821D
:101AAD00E43517F583ECF0AB18AA17AF10122061CF
:051ABD00AF10021D2323
:0321D800021A7771
:0A1D59008E348F358D368A378B38B3
:101D6300E4F539E539C3953650200535E535AE340C
:101D73007002053414FFE5382539F582E43537F56B
:0A1D830083E0FD1221D8053980D954
:011D8D002233
:0819DB007A287B007F017E1FCA
:0A19E3008E328F338D348A358B3637
:1019ED00E4FDF537E5166012E532FF7E000DEE25BC
:1019FD0018F582E43517F583EFF0AE050DE5182ED9
:101A0D00F582E43517F583E533F0AB18AA17AF105F
:0E1A1D00122061AB36AA35AD34AF1002204561
:1009860090E6BAE0752A00F52BA3E0FEEE422A9027
:10099600E6BEE0752C00F52DA3E0FEEE422C90E6B7
:1009A600B8E064C06003020A93E52D452C7003028B
:1009B6000B2690E6A0E020E1F9C3E52D9440E52C56
:1009C60094005008852C2E852D2F8006752E0075D7
:1009D6002F4090E6B9E064A3705890E6BCE0B401FD
:1009E6001BA3E0701790E6BBE030E71090E7407479
:1009F60003F0A37401F0A37403F0806CE4F530F502
:100A060031C3E531952FE530952E505CE52B253128
:100A1600F582E52A3530F583E0FF74402531F5820D
:100A260074E73530F583EFF00531E53170D30530E5
:100A360080CFE4F530F531C3E531952FE530952EBD
:100A4600501974402531F58274E73530F58374CD3D
:100A5600F00531E53170E0053080DCAD2F7AE77BBB
:100A660040AF2BAE2A1219E3E490E68AF090E68BAB
:100A7600E52FF0252BF52BE52E352AF52AC3E52D96
:100A8600952FF52DE52C952EF52C0209AF90E6B89D
:100A9600E064406003020B26E52D452C7003020B33
:100AA60026E490E68AF090E68BF090E6A0E020E15E
:100AB600F990E68BE0752E00F52F90E6B9E0B4A329
:100AC60036E4F530F531C3E531952FE530952E50F6
:100AD6003374402531F58274E73530F583E0FFE560
:100AE6002B2531F582E52A3530F583EFF00531E522
:100AF6003170D3053080CFAD2F7AE77B40AF2BAE78
:100B06002A121D59E52F252BF52BE52E352AF52A18
:100B1600C3E52D952FF52DE52C952EF52C020A9E75
:010B260022AC
:0221DE00C3221A
:0221E000D32208
:0221E200D32206
:0800030090E6BAE0F50BD322F0
:1021640090E740E50BF0E490E68AF090E68B04F00B
:02217400D32274
:0821C00090E6BAE0F511D3220C
:1021760090E740E511F0E490E68AF090E68B04F0F3
:02218600D32262
:0221E400D32204
:0221E600D32202
:0221E800D32200
:10114200E4FF90E6B8E020E70302122F0F0F74408D
:101152002401F582E434E7F583740AF00F74402425
:1011620002F582E434E7F583E4F00F74402403F5DA
:1011720082E434E7F583E4F00F74402404F582E45A
:1011820034E7F5837404F00F74402405F582E434E7
:10119200E7F5837404F00F74402406F582E434E723
:1011A200F583E4F00F74402407F582E434E7F58315
:1011B200E4F00F74402408F582E434E7F58374FF09
:1011C200F00F74402409F582E434E7F58374FFF0EC
:1011D2000F7440240AF582E434E7F5837408F00FB3
:1011E2007440240BF582E434E7F5837420F00F7425
:1011F20040240CF582E434E7F583741FF00F744049
:10120200240DF582E434E7F583741FF00F74402453
:101212000EF582E434E7F5837401F090E740EFF0D5
:0D122200E490E68AF090E6BEE090E68BF0E6
:01122F00229C
:100B270090E6B9E01206E20B6E100B6E110BB214D1
:100B37000C66150B5C280B562E0B503C0B683F0BB5
:100B470062A20B62A300000CA0120056020CA212B4
:100B57000DF0020CA2121230020CA2120986020C2E
:100B6700A2121142020CA290E6B8E030E70C7B011A
:100B77007AE7794012000E020C8A90E6BEE0701008
:100B870090E6BCE0FF90E6BAE0FD121886020CA2E0
:100B970090E6BEE090E68BF090E6A0E020E1F97BDE
:100BA700017AE77940121E86020CA2C2AF90E75085
:100BB700E515F0E4F5157B017AE7794C12000EE4B0
:100BC700F52674912526F582E43428F583E0FF7431
:100BD700402526F582E434E7F583EFF00526E52680
:100BE700B404DF90E6BCE06027E4F526749B252675
:100BF700F582E43428F583E0F4FF74442526F58272
:100C0700E434E7F583EFF00526E526B404DE802417
:100C1700E4F526749B2526F582E43428F583E0FF66
:100C270074442526F582E434E7F583EFF00526E5DD
:100C370026B404DFE4F52674972526F582E43428E4
:100C4700F583E0FF74482526F582E434E7F583EF62
:100C5700F00526E526B404DF121C7CD2AF8024E41D
:100C6700F526746D2526F582E43428F583E0FF74B4
:100C7700402526F582E434E7F583EFF00526E526DF
:100C8700B404DFE490E68AF090E6BEE090E68BF0ED
:0C0C970090E6A0E04480F08002C322D36D
:010CA300222E
:101FB200C0E0C083C08290E6B5E04401F0D2015394
:0F1FC20091EF90E65D7401F0D082D083D0E032D1
:1020FC00C0E0C083C0825391EF90E65D7404F0D0D1
:06210C0082D083D0E03216
:10211200C0E0C083C0825391EF90E65D7402F0D0BC
:0621220082D083D0E03200
:101CB500C0E0C083C08290E680E030E70E853F43F8
:101CC500854044854745854846800C85474385487A
:101CD50044853F458540465391EF90E65D7410F08D
:071CE500D082D083D0E03271
:1020E400C0E0C083C082D2035391EF90E65D7408D0
:0820F400F0D082D083D0E0326D
:101CEC00C0E0C083C08290E680E030E70E853F43C1
:101CFC00854044854745854846800C854743854843
:101D0C0044853F458540465391EF90E65D7420F045
:071D1C00D082D083D0E03239
:0121F10032BB
:0121F20032BA
:0121F30032B9
:0121F40032B8
:0121F50032B7
:0121F60032B6
:0121F70032B5
:0121F80032B4
:0121F90032B3
:0121FA0032B2
:0121FB0032B1
:0121FC0032B0
:0121FD0032AF
:0121FE0032AE
:0121FF0032AD
:0122000032AB
:0122010032AA
:0122020032A9
:0122030032A8
:0122040032A7
:0122050032A6
:0122060032A5
:0122070032A4
:0122080032A3
:0122090032A2
:01220A0032A1
:01220B0032A0
:01220C00329F
:01220D00329E
:01220E00329D
:01220F00329C
:01221000329B
:01221100329A
:012212003299
:012213003298
:012214003297
:10202900E4F5C8E58E54074438F58E8FCB8FCDAFD4
:0C203900058FCA8FCCD2BDD2ADD2CA2216
:101E2600AB07AA06A905A8047F007E1B7D377C4B5D
:101E36001204E7AB07AA06A905A804E4FFFE7D8005
:101E46007C471203EF120584AD07AC06AF040220EF
:011E56002962
:10218800AD07AC06C3E49DFBE49CFFEBFD022029F0
:0321DB00C2CA2253
:03002B00021B8B2A
:101B8B00C0E0C0F0C083C082C0D075D000C000C020
:101B9B0001C002C003C004C005C006C0071221ED7E
:101BAB00C2CFD007D006D005D004D003D002D001CD
:0D1BBB00D000D0D0D082D083D0F0D0E03266
:0A21B6000001020203030404050502
:03000B00021A2BAB
:101A2B00C0E0C0F0C0D075D000C000C004C005C07D
:101A3B0006C007053EE53EB40621051AE51A7002FD
:101A4B000519AE19FF7C007D0A12067FED4C70085C
:101A5B000513E51370020512753E00D007D006D0B2
:0C1A6B0005D004D000D0D0D0F0D0E03284
:10145500E4F524F523F522F521C203C200C202C238
:1014650001121C4075410F75422B75490F754A3D98
:10147500753F0F75404775470F754867754B0F7575
:101485004C87D2E843D82090E668E04409F090E61E
:101495005CE0443DF0D2AFD207121E5790E680E0E3
:1014A50054F7F0C203300105120761C20130032968
:1014B5001221DE5024C2031212D620001690E682B5
:1014C500E030E704E020E1EF90E682E030E604E07A
:0E14D50020E0E4121EB41221E0121FEF80C7C7
:1007610090E6B9E0700302081214700302088F24A6
:10077100FE700302091224FB700302080C147003BB
:10078100020806146073146076240560030209727E
:100791001221E2400302097E90E6BBE024FE6022C2
:1007A10014603324FD601114602224067048E54171
:1007B10090E6B3F0E5428037E54990E6B3F0E54ACB
:1007C100802DE54390E6B3F0E5448023E54590E6CE
:1007D100B3F0E546801990E6BAE0FF121EE0AA06E2
:1007E100A9077B01EA494B600DEE90E6B3F0EF906B
:1007F100E6B4F002097E02097712217602097E121F
:1008010021C002097E12000302097E12216402093D
:100811007E1221E4400302097E90E6B8E0247F6065
:100821001514601924027063A200E43325E0FFA2CD
:1008310002E4334F8041E490E740F0803F90E6BC12
:10084100E0547EFF7E00E0D394807C0040047D0173
:1008510080027D00EC4EFEED4F24B6F58274213E00
:10086100F583E493FF3395E0FEEF24A1FFEE34E638
:100871008F82F583E0540190E740F0E4A3F090E625
:100881008AF090E68B7402F002097E020977122148
:10089100E6400302097E90E6B8E024FE60162402D9
:1008A100600302097E90E6BAE0B40105C2000209C4
:1008B1007E02097790E6BAE0705590E6BCE0547E7E
:1008C100FF7E00E0D394807C0040047D0180027DA6
:1008D10000EC4EFEED4F24B6F58274213EF583E423
:1008E10093FF3395E0FEEF24A1FFEE34E68F82F50E
:1008F10083E054FEF090E6BCE05480131313541FC0
:10090100FFE0540F2F90E683F0E04420F0806E80EA
:10091100651221E8506790E6B8E024FE601A2402CF
:10092100705B90E6BAE0B40104D200805090E6BA60
:10093100E0B402028047803E90E6BCE0547EFF7E38
:1009410000E0D394807C0040047D0180027D00ECB6
:100951004EFEED4F24B6F58274213EF583E493FFFC
:100961003395E0FEEF24A1FFEE34E68F82F583801C
:1009710008120CA4500790E6A0E04401F090E6A014
:04098100E04480F0DE
:01098500224F
:030033000221D4D3
:0421D40053D8EF32BB
:101EB40090E682E030E004E020E60B90E682E03039
:101EC400E119E030E71590E680E04401F07F147EEC
:0C1ED40000121AC290E680E054FEF022DA
:1012D60090E682E044C0F090E681F043870100008A
:0412E60000000022E2
:101E570030070990E680E0440AF0800790E680E0CA
:101E67004408F07FDC7E05121AC290E65D74FFF02D
:0F1E770090E65FF05391EF90E680E054F7F02291
:0821C800E4F552D2E9D2AF2286
:101D230090E678E020E6F9C2E990E678E04480F0B6
:101D3300EF25E090E679F090E678E030E0F990E680
:101D430078E04440F090E678E020E6F990E678E029
:061D530030E1D6D2E922C6
:101DF400A90790E678E020E6F9E552702390E678AA
:101E0400E04480F0E925E090E679F08D4DAF03A938
:101E140007754E018A4F8950E4F551755201D3225A
:021E2400C322D7
:101D8E00A90790E678E020E6F9E552702590E6780E
:101D9E00E04480F0E925E0440190E679F08D4DAF06
:101DAE0003A907754E018A4F8950E4F55175520308
:041DBE00D322C32247
:03004B0002103A66
:10103A00C0E0C083C082C085C084C086758600C0F7
:10104A00D075D000C000C001C002C003C006C007EE
:10105A0090E678E030E20675520602112490E678AE
:10106A00E020E10CE5526402600675520702112481
:10107A00E55224FE605F14603624FE7003021115E7
:10108A0024FC700302112124086003021124AB4ED0
:10109A00AA4FA950AF5105518F8275830012061EBF
:1010AA0090E679F0E551654D7070755205806B9048
:1010BA00E679E0AB4EAA4FA950AE518E82758300F5
:1010CA0012065D755202E54D6401704E90E678E0B5
:1010DA004420F08045E54D24FEB5510790E678E0BE
:1010EA004420F0E54D14B5510A90E678E04440F00A
:1010FA0075520090E679E0AB4EAA4FA950AE518ED8
:10110A008275830012065D0551800F90E678E044EF
:10111A0040F075520080037552005391DFD007D01A
:10112A0006D003D002D001D000D0D0D086D084D04F
:08113A0085D082D083D0E032A1
:021EE000A90750
:101EE200AE4BAF4C8F828E83A3E064037017AD01BB
:101EF20019ED7001228F828E83E07C002FFDEC3E73
:091F0200FEAF0580DF7E007F00C8
:011F0B0022B3
:10204500121D8EE55224FA600E146006240770F303
:0C205500D322E4F552D322E4F552D3224A
:10206100121DF4E55224FA600E146006240770F381
:0C207100D322E4F552D322E4F552D3222E
:101AC2008E258F2690E600E054187012E526240138
:101AD200FFE43525C313F525EF13F526801590E6AF
:101AE20000E05418FFBF100BE52625E0F526E5259A
:101AF20033F525E5261526AE25700215254E60051F
:061B02001212EA80EE223F
:1012EA007400F58690FDA57C05A3E582458370F917
:0112FA0022D1
:03004300021300A5
:0300530002130095
:10130000021FB200022112000220FC000220E400B1
:10131000021CB500021CEC000221F1000221F200C7
:101320000221F3000221F4000221F5000221F6005F
:101330000221F7000221F8000221F9000221FA003F
:101340000221FB000221F2000221FC000221FD002B
:101350000221FE000221FF00022200000222010001
:10136000022202000221F2000221F2000221F20018
:1013700002220300022204000222050002220600CB
:1013800002220700022208000222090002220A00AB
:1013900002220B0002220C0002220D0002220E008B
:1013A00002220F000222100002221100022212006B
:0813B0000222130002221400C6
:1003EC000205F0E86480F8E933E83360110460F04A
:1003FC00ED33EC337009E8FCE9FDEAFEEBFF220477
:10040C0060DED3EB9FEA9EE99DE8C2E78CF0C2F771
:10041C0095F0400CE8CCF8E9CDF9EACEFAEBCFFB3D
:10042C001205BB85D0F05804700320D5B3E80470D6
:10043C00075002B2D50205FA92D5EC0460F7E4CC71
:10044C00C0E0C398F8603B94186008400DD0E0FB06
:10045C000205D2E4FBFAC9FC8028E830E406E4C9C2
:10046C00FBE4CAFCE830E305E4C9CACBFCE854075A
:10047C006010F8C3E913F9EA13FAEB13FBEC13FC65
:10048C00D8F130F52FC3E49CFCEF9BFFEE9AFEED08
:10049C0099FDD0E0FBEF4E4D4C701222DB030205B0
:1004AC00F7EC2CFCEF33FFEE33FEED33FDED30E7D4
:1004BC00EB0205D2EF2BFFEE3AFEED39FDD0E0FB5F
:1004CC0050130BBB00030205FAED13FDEE13FEEF08
:0804DC0013FFEC13FC0205D232
:1004E4000205FAEC5D046005E8590470030205F0A6
:1004F4001205BB580460F6EC4860F2EC7004FDFE93
:10050400FF22C860DB2481C85009C39860025006EA
:100514000205F79850CAF582E9294B4A7005AB8267
:100524000205E675F0007C1A7880C3EF9BEE9AED25
:1005340099400DC3EF9BFFEE9AFEED99FDE842F062
:10054400DC23ACF0D0E0FFD0E0FED0E0FDAB8220B5
:10055400E7101BEB60BAEC2CFCEF33FFEE33FEED3F
:1005640033FD0205D2E803F830E705C0F075F0006A
:10057400EF2FFFEE33FEED33FD40B830E7C280AA23
:10058400EDD2E7CD33EC3392D524814006E4FFFE6F
:10059400FDFC22FCE4CFCECDCC24E0501174FF80CE
:1005A400EDC3CC13CCCD13CDCE13CECF13CF04706B
:0705B400F030D5DE0206D491
:1005BB00E9D2E7C933E833F892D5EDD2E7CD33EC86
:0705CB0033FC5002B2D522FF
:1005D200EC30E7100FBF000C0EBE00080DBD00048A
:1005E2000BEB6014A2D5EB13FCED92E7FD2274FF36
:1005F200FCFDFEFF22E480F8A2D574FF13FC7D808F
:03060200E480EFA2
:030000000214E304
:0C14E300787FE4F6D8FD75815902152AC7
:10060500BB010689828A83E0225002E722BBFE02F3
:09061500E32289828A83E4932226
:10061E00BB010CE58229F582E5833AF583E0225091
:10062E0006E92582F8E622BBFE06E92582F8E222DB
:0D063E00E58229F582E5833AF583E49322F5
:10064B00BB010689828A83F0225002F722BBFE018E
:02065B00F32288
:10065D00F8BB010DE58229F582E5833AF583E8F0D3
:10066D00225006E92582C8F622BBFE05E92582C87F
:02067D00F22267
:10067F00BC000BBE0029EF8DF084FFADF022E4CC5F
:10068F00F875F008EF2FFFEE33FEEC33FCEE9DEC28
:10069F00984005FCEE9DFE0FD5F0E9E4CEFD22ED6E
:1006AF00F8F5F0EE8420D21CFEADF075F008EF2FB8
:1006BF00FFED33FD4007985006D5F0F222C398FDA9
:0506CF000FD5F0EA2246
:0E06D400C3E49FFFE49EFEE49DFDE49CFC2237
:1006E200D083D082F8E4937012740193700DA3A3A7
:1006F20093F8740193F5828883E4737402936860BB
:06070200EFA3A3A380DFBA
:10070800D083D082F8E4937012740193700DA3A380
:1007180093F8740193F5828883E473740293B5F0B7
:0D072800067403936860E9A3A3A3A380D81F
:101989008B348A358936E4F53CF53DE53B153BAEAC
:101999003A7002153A4E6033AB37AA38A9391206A4
:1019A90005FFAB34AA35A936053DE53DAC3C7002CF
:1019B900053C14F5828C83EF12065DEF60CD74014E
:1019C9002539F539E43538F53880C0AB34AA35A95D
:0219D9003622B4
:10213D00E4FFFE120605600C0FEF70010E09E97049
:05214D00F20A80EF2200
:10073500EF4E6012EF60010EEDBB010B89828A83DB
:10074500F0A3DFFCDEFA2289F05007F709DFFCA9E8
:0C075500F022BBFEFCF309DFFCA9F0223F
:1014EF00021455E493A3F8E493A34003F68001F2AA
:1014FF0008DFF48029E493A3F85407240CC8C333FE
:10150F00C4540F4420C8834004F456800146F6DFCC
:10151F00E4800B0102040810204080902128E47E13
:10152F00019360BCA3FF543F30E509541FFEE493C1
:10153F00A360010ECF54C025E060A840B8E493A388
:10154F00FAE493A3F8E493A3C8C582C8CAC583CAB3
:10155F00F0A3C8C582C8CAC583CADFE9DEE780BE6B
:01213C0000A2
:00000001FF
